:020000020000FC
:100000000FC00EC00DC00CC00BC00AC009C008C094
:1000100007C006C005C004C003C002C001C000C0C4
:1000200002C0AFD00DC06FED6DBF96988E989498BA
:100030008C9A8D98959860E1762E8D987ED041C0EF
:100040003AE302D230E200D230E2FED15ED0AF33EA
:10005000A9F0A132A9F0AF7DA23569F0AD3009F366
:10006000A134B9F0A23409F1A33459F1A434A9F1AF
:10007000A53471F0E5CF85D0E3CFE2CF5ED0E0CFFD
:10008000F2E0E8EA4FD0A89568E061BDFFCFD8CF95
:1000900030C061E0262E61E0362E64EF462E67E226
:1000A000562EF2E0E8EC3ED0CBCF61E0262E6AE09F
:1000B000362E64EF462E67E2562EF2E0EAEF32D09B
:1000C000BFCF61E0262E64E6362E64EF462E67E24F
:1000D000562EF3E0EEE226D0B3CF6AE0262E64E699
:1000E000362E64EF462E67E2562EF3E0EEE51AD088
:1000F000A7CF64E6262E64E6362E64EF462E67E22E
:10010000562EF3E0E4E90ED09BCF62D1583109F0CE
:10011000FCCF0895FADF3A2F97D10895F2E0E4EC8E
:1001200001D00895C895002021F0302D8DD1319651
:10013000F9CF0895F7DFF2DF0895F0DFEFDFF2E0A7
:10014000E6E0F8DF08954C2F46954695469546958E
:10015000405D4A3308F0495FCF70C05DCA3308F094
:10016000C95F0895F0DF342F6FD13C2F6DD1089512
:1001700068E030E3CC1F08F431E366D16A95C9F733
:10018000089560E06FBD60E06DBD6CBD66E06EBD62
:10019000122C932D742D852D7A957030E9F78A9560
:1001A0008030D1F70000000000009A9599F71A946A
:1001B00081F760E06EBD0CB51DB50CD0AFDF3F2DF3
:1001C00060E3360F41D1CE2DCDDFCD2DCBDF30E238
:1001D0003BD1089520E1FF24EE24DD24FF27000F0A
:1001E000111FDD1CEE1CFF1C2A9509F40895E0E1A7
:1001F00032913D5F33FD30833081305D37FD308398
:10020000ED30B1F7ECCF3233313320667265717562
:10021000656E6379206D65746572202032303032EE
:100220002E30362E31312041205246204C494E4B43
:10023000202020204469636B2043617070656C73DB
:100240000A0D413D31306D732C423D3130306D73BC
:100250002C433D31732C443D3130732C453D3130BE
:1002600030732E2052657475726E206F7220523D6D
:100270006D656175737265200A0D4D617820636F3D
:10028000756E74203D2036353533352C204D617820
:10029000206672657175656E6379203C2034204D4F
:1002A000487A2E200A0D00004861726477617265F9
:1002B00020726573657420696E6974696174656420
:1002C0002E2000000A0D000054696D65626173659F
:1002D0002073657420746F203130206D7320467256
:1002E000657175656E637920697320436F756E74EF
:1002F00020583130302E0A0D000054696D6562615E
:1003000073652073657420746F20313030206D73F5
:100310002E204672657175656E637920697320437E
:100320006F756E742058203130200A0D000054691A
:100330006D65626173652073657420746F20312070
:10034000732E204672657175656E6379206973201E
:10035000436F756E74205820312E0A0D00005469C9
:100360006D65626173652073657420746F20313030
:1003700020732E204672657175656E6379206973EE
:1003800020436F756E7420205820312F31302E207D
:100390000A0D000054696D656261736520736574B0
:1003A00020746F2031303020732E204672657175B5
:1003B000656E637920697320436F756E74202058D1
:1003C00020312F3130302E200A0D000050E00895EA
:1003D00050E060E0362F19D0CEF3C0F333953930BA
:1003E000D2F313D09EF3E8F768E0362F0ED076F301
:1003F000551F3A95D9F709D04EF368E0362F05D04E
:100400002EF3AA1F3A95D9F7089580E076E17A9500
:10041000F1F78395B9F08699F9CF76E17A95F1F7FE
:10042000839581F0869BF9CF823462F08E363AF064
:10043000843842F08C3D32F4E89488940895E8942E
:10044000089408956894089550E06FE0662E8894AB
:100450000DD0572D08D0532F06D05FEF62E0662EE7
:10046000089404D0089569E0662E0894949A80E078
:1004700074E008F078E08A95F1F77A95E1F79498BE
:1004800080E074E008F078E08A95F1F77A95E1F77A
:08049000551F6A9459F7089505
:00000001FF
